:030000000218DC07
:0C18DC00787FE4F6D8FD758163021923C3
:0F1F5E007D607C09ED1D70011C144C70F7DFF1E4
:011F6D002251
:0600030000007F0CDFFE8F
:0100090022D4
:05000E00007F05DFFE8C
:0100130022CA
:10102300EFD394077480948040037F0122120999BF
:10103300FED394037480948040037F0222EF7044B4
:10104300EE700B9000011209B2F4529352941209FC
:10105300996401700B9000011209B24293F4529407
:10106300120999FE6402700A9000011209B24293B8
:101073004294EE6403700D9000011209B2FEF45223
:1010830093EE4294EF64017046120999FE700B903F
:1010930000011209B2F452915292EE6401700B9066
:1010A30000011209B24291F452921209996402703A
:1010B3000A9000011209B242914292120999640303
:1010C300700D9000011209B2FEF45291EE4292EFBC
:1010D30064027046120999FE700B9000011209B266
:1010E300F452955296EE6401700B9000011209B20E
:1010F3004295F452961209996402700A9000011203
:1011030009B2429542961209996403700D90000149
:101113001209B2FEF45295EE4296EF640370461242
:101123000999FE700B9000011209B2F452B152B248
:10113300EE6401700B9000011209B242B1F452B295
:101143001209996402700A9000011209B242B14275
:10115300B21209996403700D9000011209B2FEF4F2
:1011630052B1EE42B2EF64047046120999FE700B5D
:101173009000011209B2F452B352B4EE6401700B41
:101183009000011209B242B3F452B41209996402F5
:10119300700A9000011209B242B342B41209996471
:1011A30003700D9000011209B2FEF452B3EE42B483
:1011B300EF64057046120999FE700B900001120945
:1011C300B2F452C952CAEE6401700B9000011209C5
:1011D300B242C9F452CA1209996402700A9000011A
:1011E3001209B242C942CA1209996403700D9000F0
:1011F300011209B2FEF452C9EE42CAEF6406704608
:10120300120999FE700B9000011209B2F452CB52ED
:10121300CCEE6401700B9000011209B242CBF45280
:10122300CC1209996402700A9000011209B242CBF0
:1012330042CC1209996403700D9000011209B2FEA9
:10124300F452CBEE42CCEF64077049120999FF7E4A
:1012530000700B9000011209B2F452E152E2EF6404
:10126300014E700B9000011209B242E1F452E212F6
:1012730009996402700A9000011209B242E142E244
:101283001209996403700D9000011209B2FFF45220
:07129300E1EF42E27F0022BF
:101D08007543ECE4F542FB7A0079427F0312102315
:101D180075431C7542037F011210237543E1E4F5F6
:101D2800427F01121023754310E4F5427F0512101B
:031D380023D2941F
:011D3B002285
:05001E0025640D0A003D
:10002600120014121D70121D08121E58121D3CD209
:10003600AF7F0A121F5E1200A612129A121B3A1204
:100046001E017BFF7A00791E856148856047855FC2
:0900560046855E4512069F80DD1F
:0614DF008B4E8A4F89507C
:1014E500EF640160030216D9755601F557F558F5F5
:1014F50059F55AF55BF55CFFEFC394207480948031
:10150500500F74202FF582E43400F583E4F00F804A
:10151500E7E4FFEFC3942074809480500F74002F8C
:10152500F582E43400F583E4F00F80E7AB4EAA4F73
:10153500A95090000A1209B2FD7C00D3940374806F
:10154500948040037F0222ED4C700553B7EFC2BC77
:10155500AB4EAA4FA95090000A1209B2640170055A
:1015650053B7EFD2BC90000A1209B2FF7E006402A5
:10157500700543B710C2BCEF64034E700543B71046
:10158500D2BC120999FD7C00D394C074809480402C
:10159500037F0222120999FFE598543F4FF598ED14
:1015A50064C04C6008EF6440600302166690000258
:1015B500120C297F807E8D7D5B7C00120B738F540E
:1015C5008E538D528C51E4FFFE7D01FCAB54AA5322
:1015D500A952A851C3120C0540037F0222C3E4950A
:1015E50054F554E49553F55374019552F552E49529
:1015F50051F551AB4EAA4FA9509000011209B2FB0B
:101605007A006401702CC28E538EFE5389BF5389B4
:10161500CF438E40AF54AE53AD52AC517808120C47
:10162500168F8D85548BC2AB5389BF538FFDD28ED8
:101635008069EB64024A7026538EEF438E01538E08
:10164500F7438E04AF54AE53AD52AC517808120C2B
:10165500168FD68554D753AFFB438E10803D7F023E
:1016650022AB4EAA4FA950120999FF7E0070149023
:1016750000081209B264017005438E20801D538E47
:10168500DF8018EF64804E70129000081209B26472
:10169500017005438780800353877FAB4EAA4FA90E
:1016A500509000091209B264017004D2AC8002C2E4
:1016B500AC9000071209B264017004D29C8002C28A
:1016C5009C90000B1209B254C0FFE5A2543F4FF5A0
:0616D500A27F00227F024B
:0116DB0022EC
:101E810074202558F582E43400F583EFF00558C33A
:101E9100E5589420748094804003E4F558E5597026
:071EA10005755901D29922D9
:101F3800120999FF600C121E81740129F9E43AFA1A
:031F480080EE2206
:030023000219EBD4
:1019EB00C0E0C083C082C0D075D000C0073098283B
:1019FB00C298E55C7022C3E55A94207480948040B1
:101A0B0003755A00AF5A055A74002FF582E434005F
:101A1B00F583E599F0755B0530992BC299E5576510
:101A2B0058602074202557F582E43400F583E0F5E7
:101A3B00990557C3E55794207480948040087557D7
:101A4B00008003755900D007D0D0D082D083D0E06E
:011A5B003258
:101E58007542407543017547007546C27545017561
:101E68004400754901E4F54A754B01F54CF54DFB05
:091E78007A0079427F010214DFB7
:05009E00AE07021E8107
:071BA80002620000015D0074
:03000B00021836A2
:10183600C0E0C0F0C083C082C0D075D000C000C078
:1018460001C002C003C004C005C006C007E50964A4
:101856000370277E017490A817088005C333CE3322
:10186600CED8F9FFEE3395E0FDFCAB61AA60A95F27
:10187600A85ED3120C055002C292E4FFFEFDFCAB3B
:1018860061AA60A95FA85ED3120C05500E756100AF
:10189600756000755F00755E008020E50A64017062
:1018A6001AE56124FFF561E56034FFF560E55F3414
:1018B600FFF55FE55E34FFF55EB293D007D006D044
:1018C60005D004D003D002D001D000D0D0D082D031
:0618D60083D0F0D0E032E7
:03001B0002000AD6
:01000A0032C3
:03006300021C0775
:101C0700C0E0C0D00563E56370020562C394C8E510
:101C1700629400402E309213E55D9407748094809F
:101C27004005755D008016055D8012D3E55D940063
:101C3700748094805005755D078002155D7562009C
:101C4700756300E514600A051EE51E700A051D8010
:0C1C570006751D00751E00D0D0D0E032D4
:03009B0002001A46
:01001A0032B3
:0300A30002005FF9
:01005F00326E
:100CF200AD07EDD394047480948040037F0122ED0C
:100D02006003020DC7C28C9000021209B264017026
:100D120004D2A98002C2A99000011209B2FED394A2
:100D2200037480948040037F0222EEFF7E007005F0
:100D320053B7FDC2B9EF64014E700553B7FDD2B986
:100D4200EF64024E700543B702C2B9EF64034E70FE
:100D52000543B702D2B9120999FEC3940374809471
:100D62008040037F0222E58954FC4EF589900003FE
:100D72001209B2FF7E0064017003538E7FEF4E7042
:100D820003438E80EF64024E70054389048003534F
:100D920089FB9000041209B264017005438F01803F
:100DA20003538FFE900005120AB0E5F0F58C900017
:100DB20005120AB0F58A9000071209B264017002A6
:100DC200D28C7F0022ED64016003020E94C28E90E9
:100DD20000021209B264017004D2AB8002C2AB906D
:100DE20000011209B2FED394037480948040037F01
:100DF2000222EEFF7E00700553B7F7C2BBEF64011B
:100E02004E700553B7F7D2BBEF64024E700543B77D
:100E120008C2BBEF64034E700543B708D2BB120988
:100E220099FEC394037480948040037F0222EEC42F
:100E320054F0FFE58954CF4FF5899000031209B2AF
:100E4200FF7E0064017003538EBFEF4E7003438E2A
:100E520040EF64024E700543894080035389BF907E
:100E620000041209B264017005438F028003538F9C
:100E7200FD900005120AB0E5F0F58D900005120A0A
:100E8200B0F58B9000071209B264017002D28E7F16
:100E92000022ED6402707C538EEF9000021209B2C0
:100EA2006401700543AF04800353AFFB900003124B
:100EB20009B2FED394027480948040037F0222EE32
:100EC200FF7E0064017003538EFBEF4E7003438E6E
:100ED20004EF64024E7005438E088003538EF79030
:100EE20000041209B264017005438F048003538F1A
:100EF200FB900005120AB0E5F0F5D6900005120A43
:100F0200B0F5D79000071209B264017003438E1046
:100F12007F0022ED6403707C53D1F7900002120926
:100F2200B26401700543AF20800353AFDF9000032A
:100F32001209B2FED394027480948040037F02228D
:100F4200EEFF7E006401700353D1FDEF4E70034348
:100F5200D102EF64024E700543D104800353D1FBEA
:100F62009000041209B26401700543D10180035359
:100F7200D1FE900005120AB0E5F0F5D490000512FA
:100F82000AB0F5D59000071209B26401700343D18B
:100F9200087F0022ED6404600302102053D17F9089
:100FA20000021209B26401700543AF40800353AFDF
:100FB200BF9000031209B2FD7C00D39402748094A6
:100FC2008040037F0222ED64014C700353D1DF9015
:100FD20000031209B2700343D1209000031209B238
:100FE2006402700543D140800353D1BF90000412C4
:100FF20009B26401700543D110800353D1EF900010
:1010020005120AB0FDACF0ECF5D2AF058FD390001B
:10101200071209B26401700343D1807F00227F026C
:0110220022AB
:101D7000E4F542F543754401F545F5467547FF75B1
:101D80004810754901FB7A007942FF120CF2E4F524
:101D900045F5467547A27548407549017F02020C1A
:011DA000F250
:101BAF0010223F065B4F666D7D077F6F777C395E36
:101BBF007971103201213018080000000100000077
:041BCF00080C0603F5
:0F1F6E00D2B2D2B3120003C2B3120003C2B22226
:0F1F7D00C2B2C2B3120003D2B2120003D2B32217
:020066008F49C0
:10006800C2B2E4F54AC3E54A9408748094805022E9
:10007800E54930E704D2B38002C2B3E54925E0F58B
:100088004912000ED2B212000EC2B212000E054A78
:0200980080D313
:01009A002243
:101EEA00E4F549D2B312000EA2B3E433F549D2B2F3
:0A1EFA0012000EC2B212000EAF4932
:011F040022BA
:061ECC00D2B3D2B27F5137
:101ED2008F47121F6E7F48120066121EEAAF47122A
:081EE2000066121EEA021F7DDA
:051EA800F8E6FD7F02D9
:101EAD008F478D48121F6EE54725E02468FF12000D
:0F1EBD0066121EEAAF48120066121EEA021F7D6F
:101F0500E4F542D3E542940374809480500BE4FDDC
:091F1500AF42121EAD054280EA44
:011F1E0022A0
:06001400121ECC021F05C4
:101CD2008F458D46121ECC74322546F8E6FDE4FF90
:101CE200121EAD1200037D737F01121EAD1200039E
:101CF20074222545121EA8120003743A2546F8E6FE
:061D0200FD7F03021EAD8F
:101E2E008F45121ECC7D40E4FF121EAD1200037DC5
:101E3E00737F01121EAD12000374222545121EA8D7
:0A1E4E001200037D407F03021EAD69
:101A5C008F45121ECC7D40E4FF121EAD120003D345
:101A6C00E5459463748094804012E54575F0648478
:101A7C0075F00A84742225F0F8E68001E4FD7F01FC
:101A8C00121EAD120003D3E5459409748094804076
:101A9C0012E54575F00A8475F00A84742225F0F875
:101AAC00E68001E4FD7F02121EAD120003E54575D0
:0F1ABC00F00A84742225F0F8E6FD7F03021EADC8
:101968008E458F46121ECC7D48E4FF121EAD120034
:1019780003D3E5469463E54594004019AE45AF4668
:101988007C007D64120A257C007D0A120A257422D7
:101998002DF8E68001E4FD7F01121EAD120003D38D
:1019A800E5469409E54594004019AE45AF467C00EC
:1019B8007D0A120A257C007D0A120A2574222DF858
:1019C800E68001E4FD7F02121EAD120003AE45AFB2
:1019D800467C007D0A120A2574222DF8E6FD7F0355
:0319E800021EAD2F
:101ACB008F1F121ECC7D49E4FF121EAD120003D3F3
:101ADB00E51F9463748094804012E51F75F0648455
:101AEB0075F00A84742225F0F8E68001E4FD7F018D
:101AFB00121EAD120003D3E51F940974809480402D
:101B0B0012E51F75F00A8475F00A84742225F0F82B
:101B1B00E68001E4FD7F02121EAD120003E51F7586
:0F1B2B00F00A84742225F0F8E6FD7F03021EAD58
:101BD300011400010901010A04021D0000010800AB
:101BE30001193C011A3C011B3C011C3C0115040179
:101BF3001604011704011804090B0000000000007B
:031C0300000000DE
:10178A00E50860047F6480027FF4E50A24FD604B6B
:10179A00046003021835E5147018041209DF1209EF
:1017AA0099C394647480948040057464120A017524
:1017BA001401EFFDD3E51E9DE51D9400406D7401F3
:1017CA001209DFE4F51DF51E750801120999C39483
:1017DA00647480948040547464804DE514701EAB28
:1017EA0045AA46A947041209DF120999C394087445
:1017FA0080948040057408120A01751401D3E51E0D
:10180A009FE51D94004024AB45AA46A947740112DE
:10181A0009DFE4F51DF51E750801120999C394083C
:0B182A007480948040057408120A01CD
:011835002290
:1016DC00E50860047F6480027FF4E50A24FD604C19
:1016EC00046003021789E514701974FF1209DF12E4
:1016FC000999D3940A748094805005740A120A01D3
:10170C00751401EFFDD3E51E9DE51D9400406E742C
:10171C00FF1209DFE4F51DF51E750801120999D3B6
:10172C00940A748094805055740A8049E514702092
:10173C00AB45AA46A947120999D3940074809480AA
:10174C005006E4120A01800574FF1209DF751401BA
:10175C00D3E51E9FE51D94004023E4F51DF51E7591
:10176C000801AB45AA46A947120999D39400748085
:0D177C0094805004E4020A0174FF1209DF9A
:01178900223D
:10129A0020951FE514701BAF15FE7C017D90120A84
:1012AA0013E48F618E60F55FF55ED29275090112C3
:1012BA001C6320961FE514701BAF16FE7C017D90FF
:1012CA00120A13E48F618E60F55FF55EC2927509AA
:1012DA0002121C6320972CE51470287E037420A840
:1012EA0017088005C333CE33CED8F9FFEE3395E025
:1012FA008F618E60F55FF55ED292750903751401F0
:10130A00121C6620CC15E5147011F561F560F55FC5
:10131A00F55E750904751401121C66209029E514FE
:10132A007025E50A24FE600C14600E146004240380
:10133A007012800D750A03800B750A04121C6680F0
:10134A0003750A0275140120B755E50924FE601BCE
:10135A0014602914603724037045754500754600EA
:10136A007547157B007A00791980317545007546F5
:10137A00007547167B007A00791A8020754500753A
:10138A0046007547177B007A00791B800F75450068
:10139A007546007547187B007A00791C12178A2057
:1013AA00B655E50924FE601B14602914603724032E
:1013BA0070457545007546007547157B007A0079BA
:1013CA001980317545007546007547167B007A000D
:1013DA00791A80207545007546007547177B007A93
:1013EA0000791B800F7545007546007547187B000C
:1013FA007A00791C1216DC20B577E5147073E50AB9
:10140A0064016005750A018003750A04121C667579
:10141A001401E50924FE6019146037240270527E13
:10142A00017490A815088005C333CE33CED8F9804D
:10143A00317E017490A816088005C333CE33CED806
:10144A00F9FFEE3395E08F618E60F55FF55EC2922B
:10145A00801F7E037420A817088005C333CE33CEBD
:10146A00D8F9FFEE3395E08F618E60F55FF55ED2B5
:10147A00923096047F0180027F003095047E0180BD
:10148A00027E00EE5FFF3097047E0180027E00EE4E
:10149A005FFF30CC047E0180027E00EE5FFF309059
:1014AA00047E0180027E00EE5FFF30B7047E018079
:1014BA00027E00EE5FFF30B6047E0180027E00EEFF
:1014CA005FFF30B5047E0180027E00EE5F6005E4B6
:0514DA00F514F50822E5
:101DD2008F428C438D44E50A24FE60111460131473
:101DE200601724037018AD5DAF09021CD2AF420226
:0F1DF2001A5CAF44AE43021968AF09121E2E22CD
:101B3A00E50924FE60211460351460492403705DB0
:101B4A007E007401A815088005C333CE33CED8F9B8
:101B5A00FDAC06AF1980437E007401A81608800503
:101B6A00C333CE33CED8F9FDAC06AF1A802C7E0033
:101B7A007401A817088005C333CE33CED8F9FDAC5B
:101B8A0006AF1B80157E007401A818088005C333B0
:0E1B9A00CE33CED8F9FDAC06AF1C121DD22200
:1000A600E50924FE700302024A1470030203961443
:1000B60070030204E22403600302063CE51975F0AE
:1000C60014A4FBAAF07E007401A815088005C333AA
:1000D600CE33CED8F9FDAC06AF03AE02120A137CBE
:1000E600007D03120A7AC3EF9490EE940140030256
:1000F6000194538E7FAF197E007C007D50120C59FF
:10010600C004C005C006C0077E007401A81508809B
:1001160005C333CE33CED8F9FFEE3395E0FDFCD0E0
:1001260003D002D001D000120AE8A804A905AA0645
:10013600AB077F007E367D6E7C01120B73C3E49F96
:10014600FFE49EFE74019DFDE49CFCE4FB7A01F94C
:10015600F8120B738F8CAF197E007C007D50120C49
:1001660059C004C005C006C0077E007401A8150862
:100176008005C333CE33CED8F9FFEE3395E0FDFCD0
:10018600D003D002D001D000120AE802023F438E0B
:1001960080AF197E007C007D14120C59C004C00586
:1001A600C006C0077E007401A815088005C333CEBB
:1001B60033CED8F9FFEE3395E0FDFCD003D002D064
:1001C60001D000120AE8E47B03FAF9F8120B73A8CF
:1001D60004A905AA06AB077F007E367D6E7C011258
:1001E6000B73C3E49FFFE49EFE74019DFDE49CFC3B
:1001F600E4FB7A01F9F8120B738F8CAF197E007C41
:10020600007D14120C59C004C005C006C0077E004C
:100216007401A815088005C333CE33CED8F9FFEE96
:100226003395E0FDFCD003D002D001D000120AE8DD
:10023600E47B03FAF9F8120B73A804A905AA06AB26
:100246000702062BE51A75F014A4FBAAF07E0074CB
:1002560001A816088005C333CE33CED8F9FDAC0607
:10026600AF03AE02120A137C007D03120A7AC3EFB3
:100276009490EE94014003020304538E7FE51A75B1
:10028600F050A4FBAAF07E007401A816088005C3EE
:1002960033CE33CED8F9FDAC06AF03AE02120A1345
:1002A600AB07AA06EA3395E0F9F87F007E367D6E45
:1002B6007C01120B73C3E49FFFE49EFE74019DFD57
:1002C600E49CFCE4FB7A01F9F8120B738F8CE51AB7
:1002D60075F050A4FBAAF07E007401A816088005EC
:1002E600C333CE33CED8F9FDAC06AF03AE02120A45
:1002F60013AB07AA06EA3395E0F9F802062B438EFC
:1003060080E51A75F014A4FBAAF07E007401A81605
:10031600088005C333CE33CED8F9FDAC06AF03AEA5
:1003260002120A137C007D03120A7AAB07AA06EAB8
:100336003395E0F9F87F007E367D6E7C01120B73F3
:10034600C3E49FFFE49EFE74019DFDE49CFCE4FB78
:100356007A01F9F8120B738F8CE51A75F014A4FB69
:10036600AAF07E007401A816088005C333CE33CEEA
:10037600D8F9FDAC06AF03AE02120A137C007D036A
:10038600120A7AAB07AA06EA3395E0F9F802062BB9
:10039600E51B75F014A4FBAAF07E007401A81708EB
:1003A6008005C333CE33CED8F9FDAC06AF03AE021B
:1003B600120A137C007D03120A7AC3EF9490EE941E
:1003C600014003020450538E7FE51B75F050A4FBD9
:1003D600AAF07E007401A817088005C333CE33CE79
:1003E600D8F9FDAC06AF03AE02120A13AB07AA0694
:1003F600EA3395E0F9F87F007E367D6E7C01120BBC
:1004060073C3E49FFFE49EFE74019DFDE49CFCE43F
:10041600FB7A01F9F8120B738F8CE51B75F050A46B
:10042600FBAAF07E007401A817088005C333CE33FB
:10043600CED8F9FDAC06AF03AE02120A13AB07AA7B
:1004460006EA3395E0F9F802062B438E80E51B7524
:10045600F014A4FBAAF07E007401A817088005C357
:1004660033CE33CED8F9FDAC06AF03AE02120A1373
:100476007C007D03120A7AAB07AA06EA3395E0F9F7
:10048600F87F007E367D6E7C01120B73C3E49FFFFE
:10049600E49EFE74019DFDE49CFCE4FB7A01F9F800
:1004A600120B738F8CE51B75F014A4FBAAF07E006B
:1004B6007401A817088005C333CE33CED8F9FDAC36
:1004C60006AF03AE02120A137C007D03120A7AAB52
:1004D60007AA06EA3395E0F9F802062BE51C75F043
:1004E60014A4FBAAF07E007401A818088005C33383
:1004F600CE33CED8F9FDAC06AF03AE02120A137C9A
:10050600007D03120A7AC3EF9490EE940140030231
:10051600059C538E7FE51C75F050A4FBAAF07E0067
:100526007401A818088005C333CE33CED8F9FDACC4
:1005360006AF03AE02120A13AB07AA06EA3395E02A
:10054600F9F87F007E367D6E7C01120B73C3E49F43
:10055600FFE49EFE74019DFDE49CFCE4FB7A01F938
:10056600F8120B738F8CE51C75F050A4FBAAF07E75
:10057600007401A818088005C333CE33CED8F9FD20
:10058600AC06AF03AE02120A13AB07AA06EA33950E
:10059600E0F9F802062B438E80E51C75F014A4FBE7
:1005A600AAF07E007401A818088005C333CE33CEA6
:1005B600D8F9FDAC06AF03AE02120A137C007D0328
:1005C600120A7AAB07AA06EA3395E0F9F87F007EAD
:1005D600367D6E7C01120B73C3E49FFFE49EFE74AE
:1005E600019DFDE49CFCE4FB7A01F9F8120B738F84
:1005F6008CE51C75F014A4FBAAF07E007401A81803
:10060600088005C333CE33CED8F9FDAC06AF03AEB2
:1006160002120A137C007D03120A7AAB07AA06EAC5
:100626003395E0F9F87F007E367D6E7C01120B7300
:07063600C3E49FFF8F8A223D
:101E0100E50A24FE602314602014601D2403701C65
:101E1100E4FFFEFDFCAB61AA60A95FA85EC3120CE2
:0D1E2100057003750A04C29422D294222297
:101D3C007B007A00790B7547007548097F047E009B
:101D4C00121DA1E50BF4601B850B19850C1A850D72
:101D5C001B850E1C850F15851016851117851218FD
:041D6C0085130922B0
:031C6300751401F4
:101C66007F047E00121F4B85190B851A0C851B0DF0
:101C7600851C0E85150F851610851711851812857A
:101C860009137B007A00790B7547007548097F04B4
:051C96007E00021C9B12
:0E1F8C00E4F5C7F5C5F5C675C3FF75C4FF22A1
:061F1F008CC3AF058FC466
:101F2500A2AF92D5C2AF75C65A75C6A50000A2D597
:031F350092AF2246
:101DA100AD07AC0675C78075F51875C501121F1F03
:101DB100E5C2120A010DBD00010C740129F9E43AD2
:101DC100FAE54815487002154714454770DF021FB0
:011DD1008C85
:101F4B00AD07AC0675C78075F51875C503121F1F55
:031F5B00021F8CD6
:101C9B00AD07AC0675C78075F51875C5028CC3AF5B
:101CAB00058FC4120999F5C2121F250DBD00010C39
:101CBB00740129F9E43AFAE54815487002154714FE
:071CCB00454770D9021F8C90
:1018E800020026E493A3F8E493A34003F68001F2F0
:1018F80008DFF48029E493A3F85407240CC8C33301
:10190800C4540F4420C8834004F456800146F6DFCF
:10191800E4800B0102040810204080901BA8E47E9C
:10192800019360BCA3FF543F30E509541FFEE493C4
:10193800A360010ECF54C025E060A840B8E493A38B
:10194800FAE493A3F8E493A3C8C582C8CAC583CAB6
:10195800F0A3C8C582C8CAC583CADFE9DEE780BE6E
:011C060000DD
:10099900BB010689828A83E0225002E722BBFE025C
:0909A900E32289828A83E493228F
:1009B200BB010CE58229F582E5833AF583E02250FA
:1009C20006E92582F8E622BBFE06E92582F8E22244
:0D09D200E58229F582E5833AF583E493225E
:1009DF00BB010989828A83F8E028F022500327F7A8
:1009EF0022BBFE05F8E328F3228A838982F8E49379
:0209FF002822AC
:100A0100BB010689828A83F0225002F722BBFE01D4
:020A1100F322CE
:100A1300EF8DF0A4A8F0CF8CF0A428CE8DF0A42EF7
:020A2300FE22B1
:100A2500BC000BBE0029EF8DF084FFADF022E4CCB5
:100A3500F875F008EF2FFFEE33FEEC33FCEE9DEC7E
:100A4500984005FCEE9DFE0FD5F0E9E4CEFD22EDC4
:100A5500F8F5F0EE8420D21CFEADF075F008EF2F0E
:100A6500FFED33FD4007985006D5F0F222C398FDFF
:050A75000FD5F0EA229C
:100A7A00C2D5EC30E709B2D5E4C39DFDE49CFCEE97
:100A8A0030E715B2D5E4C39FFFE49EFE120A25C3E0
:100A9A00E49DFDE49CFC8003120A2530D507C3E4DB
:060AAA009FFFE49EFE2206
:100AB000BB0110E58229F582E5833AF583E0F5F084
:100AC000A3E0225009E92582F886F008E622BBFE61
:100AD0000AE92582F8E2F5F008E222E5832AF583A7
:080AE000E993F5F0A3E993226C
:100AE800E88FF0A4CC8BF0A42CFCE98EF0A42CFCAD
:100AF8008AF0EDA42CFCEA8EF0A4CDA8F08BF0A42B
:100B08002DCC3825F0FDE98FF0A42CCD35F0FCEB89
:100B18008EF0A4FEA9F0EB8FF0A4CFC5F02ECD394E
:0F0B2800FEE43CFCEAA42DCE35F0FDE43CFC22BB
:100B370075F008758200EF2FFFEE33FECD33CDCC75
:100B470033CCC58233C5829BED9AEC99E5829840F8
:100B57000CF582EE9BFEED9AFDEC99FC0FD5F0D6D5
:100B6700E4CEFBE4CDFAE4CCF9A88222B800C1B9FF
:100B77000059BA002DEC8BF084CFCECDFCE5F0CB3D
:100B8700F97818EF2FFFEE33FEED33FDEC33FCEB76
:100B970033FB10D703994004EB99FB0FD8E5E4F931
:100BA700FA227818EF2FFFEE33FEED33FDEC33FC1E
:100BB700C933C910D7059BE99A4007EC9BFCE99A12
:100BC700F90FD8E0E4C9FAE4CCFB2275F010EF2F57
:100BD700FFEE33FEED33FDCC33CCC833C810D70757
:100BE7009BEC9AE899400AED9BFDEC9AFCE899F892
:0E0BF7000FD5F0DAE4CDFBE4CCFAE4C8F92225
:100C0500EB9FF5F0EA9E42F0E99D42F0E89C45F045
:010C150022BC
:100C1600E8600FECC313FCED13FDEE13FEEF13FFBC
:030C2600D8F122E0
:100C2900BB010DE58229F582E5833AF583020C9330
:100C39005007E92582F8020C86BBFE07E92582F8F0
:100C4900020C9FE58229F582E5833AF583020CAC13
:100C5900EC8EF0A4CCC5F0CCCDF8EFA4CEC5F02D28
:100C6900FDE43CFCE8A42EC8C5F03DFDE43CFCEFE6
:0D0C7900A4FFE5F028FEE43DFDE43CFC2274
:10063D00E5512445F8E60551227842300702784508
:10064D00E475F001120CBC0209992000EB7F2ED24B
:10065D00008018EF540F2490D43440D4FF30040B95
:10066D00EF24BFB41A0050032461FFE55260021558
:10067D00520555E5557002055430070D7842E47565
:10068D00F001120CBCEF020A0102009E7403D207A6
:10069D008003E4C207F5518B428A438944E4F55245
:1006AD00F554F555E55260077F2012067880F575F3
:1006BD0053FFC201C200C202C203C205C206C20874
:1006CD00120646FF700D3007057F00120689AF55E3
:1006DD00AE5422B4255FC2D5C204120646FF24D003
:1006ED00B40A00501A75F00A785230D50508B6FFD5
:1006FD000106C6A426F620D5047002D20380D924A3
:10070D00CFB41A00EF5004C2E5D204020889D20119
:10071D0080C6D20080C0D20280BCD2D580BAD205AC
:10072D0080B47F201206782002077401B552004074
:10073D00F112063DFF1206780206B1D208D20680EC
:10074D009512063DFB12063DFA12063DF94A4B7015
:10075D0006795A7A097BFF20022EE552602A7E0027
:10076D008E827583001209B260060EEE655370F02D
:10077D00C2D5EBC0E0EAC0E0E9C0E0EE1208D0D08F
:10078D00E0F9D0E0FAD0E0FB120999FF60AAEBC0C6
:10079D00E0EAC0E0E9C0E0120678D0E02401F9D02B
:1007AD00E03400FAD0E0FBE5530460DCD553D9808A
:1007BD00877BFF7A0879CCD202809C7910800279F0
:1007CD0008C206C2088008D2D5790A8004790AC207
:1007DD00D5E553047002F553E4FAFDFEFF12063D14
:1007ED00FC7B0820011312063DFD7B1030000A1220
:1007FD00063DFE12063DFF7B20EC3382D592D5508F
:10080D0013C3E43000069FFFE49EFEE42001039D28
:10081D00FDE49CFCE4CBF8C201EC700CCFCECDCC4A
:10082D00E824F8F870F38017C3EF33FFEE33FEEDD5
:10083D0033FDEC33FCEB33FB994002FB0FD8E9EBB6
:10084D00300105F8D0E0C448B201C0E00AEC4D4ECD
:10085D004F78207B0070C2EAB5530040BCC0E01257
:10086D0008D2D0F0D0E0200104C4C0E0C4B201C071
:10087D00F0120661D0F0D5F0EB0206B1120CCC07E8
:10088D004E5307C858071F4C071B4207CC4F07D4C0
:0F089D004407D44907344307DA5507BE4607BE60
:1008AC004507BE47097A5007232D07272E074A2BE9
:1008BC00072B2307482009632A06E3480000074258
:1008CC003F3F3F00790AA2D5200314300509B91027
:1008DC00020404B9080104A2D52006025001042028
:1008EC0002689202B552005034C0E07F20300319E8
:1008FC007F30A20272067205500F120929C202C281
:10090C0006C205C2087F30800F300503E9C0E01233
:10091C000678300503D0E0F9D0E0B552CC3005179D
:10092C007F30B9100C1206787F583004077F78801E
:10093C0003B908031206783002057F2D0206787F72
:10094C00202008F87F2B2006F322920280CF286EFD
:10095C00756C6C2900D20112063D3001F8C2017889
:10096C005230D50108F60206E32D504349581206C1
:10097C003D2403B405004001E49009759312066907
:0D098C00743A120669D2037552040207C8BE
:0D0C8600E6FB08E6F908E6FA08E6CBF822DE
:0C0C9300E0F8A3E0F9A3E0FAA3E0FB22E4
:0D0C9F00E2FB08E2F908E2FA08E2CBF822D5
:100CAC00E493F8740193F9740293FA740393FB229E
:100CBC00FAE6FB0808E6F925F0F618E6CA3AF62239
:100CCC00D083D082F8E4937012740193700DA3A3B7
:100CDC0093F8740193F5828883E4737402936860CB
:060CEC00EFA3A3A380DFCB
:00000001FF
